:100000000C943E000C9453000C9453000C94530039
:100010000C9453000C9453000C9453000C94530014
:100020000C9453000C9453000C9453000C94530004
:100030000C9453000C9453000C9453000C945300F4
:100040000C9453000C9453000C9453000C945300E4
:100050000C9453000C9453000C9453000C945300D4
:100060000C9453000C9453000C9453000C945300C4
:100070000C9453000C9453000C94530011241FBE95
:10008000CFEFD0E1DEBFCDBF12E0A0E0B1E0E2E013
:10009000F2E002C005900D92A230B107D9F70E949C
:1000A000B4000C94FF000C940000DF93CF93CDB705
:1000B000DEB782E290E0FC01108285E290E021E070
:1000C000FC01208388E290E02FEFFC0120838BE28B
:1000D00090E0FC01108281E290E0FC01108284E259
:1000E00090E021E0FC01208387E290E02FEFFC010B
:1000F00020838AE290E0FC011082CF91DF91089585
:100100001F93DF93CF9300D00F92CDB7DEB78B83D1
:10011000809100029B8189238B838B81882F90E0C3
:1001200080509F4FFC01808189838981182F012E87
:1001300012951025012E1695169510251A838A8181
:10014000882F90E001969595879581709070009723
:1001500019F489818064898389810F900F900F90B1
:10016000CF91DF911F9108950F931F93DF93CF934A
:1001700000D0CDB7DEB70E94550085E290E025E2C1
:1001800030E0F90120812E7FFC0120831A82198240
:1001900089819A81009719F583E290E0FC018081C2
:1001A000882F90E081709070009761F485E290E074
:1001B00025E230E0F90120812160FC012083FC016F
:1001C00080810BC085E290E025E230E0F9012081DA
:1001D0002E7FFC012083FC0180811A82198208E2B3
:1001E00010E080E290E0FC0180810E948000F80134
:1001F000808389819A8101969A838983C9CFF894F3
:02020000FFCF2E
:1002020000010203040506070809242527282922DC
:1002120010131415161718121821111B321D1E1F48
:100222002334353637383933282D2A2B2C2D2E1DE1
:1002320031313A333C3536373819263B3C3D3E3F67
:10024200404142434445464748494A4B4C4D4E4F34
:10025200505152535455565758595A5B5C5D5E5F24
:10026200606162636465666768696A6B6C6D6E6F14
:10027200707172737475767778797A7B7C7D7E7F04
:10028200808182838485868788898A8B8C8D8E8FF4
:10029200909192939495969798999A9B9C9D9E9FE4
:1002A200A0A1A2A3A4A5A6A7A8A9AAABACADAEAFD4
:1002B200B0B1B2B3B4B5B6B7B8B9BABBBCBDBEBFC4
:1002C200C0C1C2C3C4C5C6C7C8C9CACBCCCDCECFB4
:1002D200D0D1D2D3D4D5D6D7D8D9DADBDCDDDEDFA4
:1002E200E0E1E2E3E4E5E6E7E8E9EAEBECEDEEEF94
:1002F200F0F1F2F3F4F5F6F7F8F9FAFBFCFDFEFF84
:020302003F00BA
:00000001FF
